:100000000C943B020C9463020C9463020C94460D16
:100010000C94210D0C94FC0C0C9463020C94630260
:100020000C9463020C9463020C9463020C946302BC
:100030000C9463020C9463020C9463020C946302AC
:100040000C94B9110C9463020C94F1030C94CB033F
:100050000C9463020C9463020C9463020C9463028C
:100060000C9463020C946302A713A315A315B91390
:100070001914A315A315D414D714A315E914A315A3
:10008000A315A315A315A315A3150515081571151B
:10009000A31583154572726F723A20004A756C2061
:1000A000203920323031392031383A34353A32353E
:1000B0000020636F6D70696C656420004E414E4F87
:1000C00000206F6E200041726475436F756E746519
:1000D000722056332E3230002000200020004900CC
:1000E00020005400206D696E20002070756C6C75C6
:1000F0007000202D002066616C6C696E67002072B4
:100100006973696E6700500040002F0073002C2057
:1001100000200048002041002053002058002C00FF
:10012000204E002054002F002044002043005200A5
:1001300056002C002042002C0020540020617661E3
:10014000696C61626C65002C002048656C6C6F2CDA
:100150002070696E7320004D20726573746F726930
:100160006E6720636F6E6669672066726F6D2045EB
:100170004550524F4D004D20696C6C6567616C2095
:10018000636F6E66696720696E20454550524F4D1A
:10019000004D206E6F20636F6E66696720696E2068
:1001A000454550524F4D002C002C002C0020004D96
:1001B00020536C6F743A200020536C6F74733A2094
:1001C000004D20454550524F4D20436F6E66696784
:1001D0003A20004D20696C6C6567616C20636F6E1E
:1001E00066696720696E20454550524F4D004D208D
:1001F0006E6F20636F6E66696720696E204545509B
:10020000524F4D00206D696C6C697365636F6E644D
:1002100073004D204E657874207265706F72742083
:10022000696E20002C200056004D205374617475B7
:10023000733A2000616C697665002C2000636F6E54
:100240006669672073617665642C20004D207265B5
:100250006D6F766564200052656D496E7400496C5F
:100260006C6567616C2070696E2073706563696688
:1002700069636174696F6E20004D20696C6C6567FD
:10028000616C2076616C75652070617373656420A4
:10029000666F7220646576566572626F7365004D95
:1002A00020646576566572626F736520736574208D
:1002B000746F20002073697A6520002C0044206749
:1002C0006F742000202072656A656374200020200E
:1002D000636F756E742000202068697374496478B8
:1002E000200020746F2000202920002C20696E74CB
:1002F00065726E616C20002028696E64657820004C
:100300004D2070696E200020616E642074726967F0
:100310006765725374617465004D2063616C6C6530
:100320006420646F436F756E742077697468207001
:10033000696E496E64657820002C2072656A656379
:100340007420002C20636F756E7420002C20686967
:1003500073744964782000206368616E6765642067
:10036000746F200029002028696E7465726E616CBC
:1003700020004D2070696E20002D3E002C004C00A6
:1003800000000000240027002A00000000002500D3
:1003900028002B00000000080002010000030407F1
:1003A000000000000000000001020408102040804E
:1003B0000102040810200102040810204D20646589
:1003C00066696E65642000416464496E7400496C1E
:1003D0006C6567616C2070756C7365206C65766503
:1003E0006C2073706563696669636174696F6E2000
:1003F000666F722070696E200000000000230026E6
:100400000029000404040404040404020202020299
:1004100002030303030303496C6C6567616C20707E
:10042000696E2073706563696669636174696F6E74
:10043000200020004D20616E616C6F67207468722F
:100440006573686F6C64732073657420746F20002B
:1004500073697A65002000200020004D20696E74C9
:10046000657276616C732073657420746F200073FD
:10047000697A6500031211241FBECFEFD8E0DEBFFA
:10048000CDBF11E0A0E0B1E0E6EBF3E302C00590E0
:100490000D92A639B107D9F726E0A6E9B1E001C06F
:1004A0001D92A938B207E1F712E0CBE3D2E004C015
:1004B0002197FE010E94AB19CA33D107C9F70E94E8
:1004C00030120C94D9190C940000CF92DF92EF9265
:1004D000FF920F931F93CF93DF936C017A018B01EF
:1004E000C0E0D0E0CE15DF0581F0D8016D918D011F
:1004F000D601ED91FC910190F081E02DC6010995A6
:10050000892B11F02196EECF7E01C701DF91CF91AB
:100510001F910F91FF90EF90DF90CF900895089575
:1005200080E090E00895FC01538D448D252F30E04C
:10053000842F90E0821B930B541710F0CF960895F0
:1005400001970895FC01918D828D981761F0828D3D
:10055000DF01A80FB11D5D968C91928D9F5F9F73F7
:10056000928F90E008958FEF9FEF0895FC01918D99
:10057000828D981731F0828DE80FF11D858D90E006
:1005800008958FEF9FEF0895FC01918D228D892FA3
:1005900090E0805C9F4F821B91098F73992708958B
:1005A00089E595E00E94C40221E0892B09F420E04E
:1005B000822F0895FC01848DDF01A80FB11DA35A7D
:1005C000BF4F2C91848D90E001968F739927848F73
:1005D000A689B7892C93A089B1898C918370806496
:1005E0008C93938D848D981306C00288F389E02D37
:1005F00080818F7D80830895EF92FF920F931F93E8
:10060000CF93DF93EC0181E0888F9B8D8C8D9813C5
:1006100005C0E889F989808185FD26C0F62E0B8DFD
:1006200010E00F5F1F4F0F731127E02E8C8DE81223
:100630000CC00FB607FCFACFE889F989808185FFE5
:10064000F5CFCE010E94DA02F1CF8B8DFE01E80FCB
:10065000F11DE35AFF4FF0829FB7F8940B8FEA89A0
:10066000FB89808180620AC09FB7F894EE89FF8978
:100670006083E889F98980818370806480839FBF6B
:1006800081E090E0DF91CF911F910F91FF90EF906B
:100690000895CF93DF93EC01888D8823C9F0EA8910
:1006A000FB89808185FD05C0A889B9898C9186FD6B
:1006B0000FC00FB607FCF5CF808185FFF2CFA88968
:1006C000B9898C9185FFEDCFCE010E94DA02E7CF88
:1006D000DF91CF91089580E090E0892B29F00E946E
:1006E000D00281110C9400000895DC01ED91FC9181
:1006F0000190F081E02D0994EF92FF920F931F93E8
:10070000CF93DF938C017B01C0E0D0E0F701EC0FC9
:10071000FD1F6491662361F0D801ED91FC91019079
:10072000F081E02DC8010995892B11F02196EECFBB
:10073000CE01DF91CF911F910F91FF90EF9008951F
:100740006115710579F0FB0101900020E9F73197FF
:10075000AF01461B570BDC01ED91FC910280F38148
:10076000E02D099480E090E0089562E971E00C9436
:10077000A0030F931F93CF93DF93EC010E947C03A0
:100780008C01CE010E94B503800F911FDF91CF91A4
:100790001F910F9108951F920F920FB60F9211247F
:1007A0002F933F934F935F936F937F938F939F9379
:1007B000AF93BF93EF93FF9389E595E00E94DA0230
:1007C000FF91EF91BF91AF919F918F917F916F9129
:1007D0005F914F913F912F910F900FBE0F901F90FF
:1007E00018951F920F920FB60F9211242F938F938B
:1007F0009F93EF93FF93E0916905F0916A058081E3
:10080000E0916F05F091700582FD12C0908180919A
:1008100072058F5F8F7320917305821751F0E091FD
:100820007205F0E0E75AFA4F958F8093720501C088
:100830008081FF91EF919F918F912F910F900FBE2B
:100840000F901F9018950C945F19CF93DF93EC01D4
:100850009C01220F331FF901E65BF94F8FEF9FEFE9
:1008600091838083FE01E059FB4F1082F901E15032
:10087000FA4F11821082CE01880F991F880F991F9D
:10088000FC01EF54FB4F1082118212821382FE0191
:10089000E25AFB4F1082FC01EA5EFB4F108211828C
:1008A00012821382F901E357FB4F11821082F90182
:1008B000EE50FC4F11821082FC01E655FC4F408344
:1008C000518362837383FC01EE59FC4F4083518353
:1008D00062837383FC01E65EFC4F40835183628335
:1008E0007383FC01E45FFA4F408351836283738317
:1008F000FE01E85FFC4F1082FE01E05DFE4F80814B
:10090000811107C0F901EE5BFE4F80810E94EC0F60
:1009100001C080E0FE01EA50FD4F8083C650DB4FEE
:100920008883DF91CF910895CF92DF92EF92FF926B
:100930000F931F93CF93DF930E948B106B017C0169
:10094000C0E0D0E0B701A601CE010E9425042196A7
:10095000C231D105B9F7C0925405D0925505E09245
:100960005605F092570510925805EDEFF3E0A5916A
:10097000B4918C9180934706EFEFF3E0A591B49189
:100980008C9180934806E1E0F4E0A591B4918C91BC
:100990008093490680E090E00E942304833461F450
:1009A00081E090E00E942304863631F482E090E0FA
:1009B0000E942304873609F161E971E089E595E039
:1009C0000E94B9030E948B10609384047093850485
:1009D0008093860490938704809188049091890481
:1009E0009093830480938204DF91CF911F910F91A4
:1009F000FF90EF90DF90CF90089583E090E00E9409
:100A00002304F82E8FEF8F0D833118F066E771E025
:100A1000D5CF67E571E089E595E00E94B903C4E0B0
:100A2000D0E010E064E0E62ECE010E942304082FFF
:100A3000CE0101960E942304D82ECE0102960E9478
:100A4000230490E0982F88278D0D911D90936F06B9
:100A500080936E06CE0103960E942304D82ECE0109
:100A600004960E94230490E0982F88278D0D911DF5
:100A70009093710680937006CE0105960E94230420
:100A8000D82ECE0106960E94230490E0982F882746
:100A90008D0D911D9093730680937206CE0107967B
:100AA0000E942304D82ECE0108960E94230490E0D1
:100AB000982F88278D0D911D90937506809374064D
:100AC0002996E0928C04093421F484E00E94820E7D
:100AD0000BC0043521F484E00E94470F05C00134A7
:100AE00019F484E00E9497101F5FF1129DCF1092BD
:100AF0008C0410928B0410928A04EEE6F6E08EE7E6
:100B000096E0119211928E179F07D9F75BCFFF9253
:100B10000F931F93CF93DF93EC01F62E0881198179
:100B2000C8010E9423048F1521F06F2DC8010E9477
:100B3000671988819981019699838883DF91CF9184
:100B40001F910F91FF900895AF92BF92CF92DF92C5
:100B5000EF92FF920F931F93CF93DF93EC015A0113
:100B600069010E9487056A2DCE010E9487056B2DC1
:100B7000CE010E9487056C2DCE010E9487056D2D48
:100B8000CE010E948705602FCE010E948705612F4C
:100B9000CE010E9487056E2DCE010E9487056F2D24
:100BA000CE01DF91CF911F910F91FF90EF90DF90D9
:100BB000CF90BF90AF900C9487052F923F924F92A9
:100BC0005F926F927F928F929F92AF92BF92CF92DD
:100BD000DF92EF92FF920F931F93CF93DF93CDB7E6
:100BE000DEB7A1970FB6F894DEBF0FBECDBF1C01D4
:100BF0006D8BF8942C01440C551C440C551C5D8ED7
:100C00004C8E820106551C4FD801CD90DD90ED90A1
:100C1000FC90CD82DE82EF82F886F201EE59FC4F25
:100C200040805180628073804E8E5F8E68A279A270
:100C3000EC8DFD8DEF54FB4FC080D180E280F380BE
:100C4000C982DA82EB82FC822C01440C551CF20131
:100C5000E357FB4F60817181FC01E25AFB4F7080CA
:100C6000EC8DFD8DE255FD4FC080D180E280F38098
:100C7000CE8ADF8AE88EF98E78948E8C9F8CA8A01D
:100C8000B9A08D819E81AF81B885881A990AAA0A78
:100C9000BB0AEC8DFD8DEA5EFB4FC080D180E28007
:100CA000F38089819A81AB81BC818C199D09AE0941
:100CB000BF0989879A87AB87BC876C017D01C718FC
:100CC000D108E108F108F201EE50FC4F80819181DA
:100CD0002B01481A590A5B8E4A8E5D885110DFC07D
:100CE000EC8DFD8DE45FFA4F80819181A281B3810B
:100CF0008D879E87AF87B88B40900A0150900B017B
:100D000060900C0170900D01498A5A8A6B8A7C8A26
:100D1000DA01C90184199509A609B7094D845E84D1
:100D20006F84788884199509A609B709B7FD47C06B
:100D30008091040190910501A0E0B0E0C816D906A9
:100D4000EA06FB06F8F08091060190910701A09158
:100D50000801B091090188159905AA05BB0590F411
:100D600080910E0190910F01A0911001B09111019D
:100D700049885A886B887C88481659066A067B061B
:100D800009F051C0F894EC8DFD8DE655FC4F2083A1
:100D9000318342835383EC8DFD8DEE59FC4F2083CC
:100DA000318342835383789449015A014D805E8098
:100DB0006F80788484189508A608B7083FC0809192
:100DC0000E0190910F01A0911001B0911101290124
:100DD0003A01481A590A6A0A7B0AD301C2014D84B2
:100DE0005E846F84788884199509A609B709B7FDD0
:100DF00037C18091040190910501A0E0B0E0C816D0
:100E0000D906EA06FB0608F42BC1809106019091F1
:100E10000701A0910801B091090188159905AA055B
:100E2000BB0508F01DC1F8948E8D9F8DA8A1B9A1B6
:100E3000F80180839183A283B3837894F894F101BD
:100E4000E25AFB4F1082EC8DFD8DE255FD4F108272
:100E50001182128213827894EC8DFD8DEA5EFB4F35
:100E600049805A806B807C8040825182628273828A
:100E7000F101EE0FFF1FEE50FC4F718360838C8DEC
:100E80009D8D845F9A4FDC012D933D934D935C9330
:100E90001397F101E85FFC4F80818F5F8083290108
:100EA0003A011D893E822D826EE271E080917E06BC
:100EB00090917F060E947C03ED81FE81EE0FFF1F63
:100EC000E65BF94F6081718180917E0690917F068B
:100ED0000E94510E6BE271E080917E0690917F0638
:100EE0000E947C0349815A816B817C8180917E06BE
:100EF00090917F060E94040E68E271E080917E0668
:100F000090917F060E947C03B701A60180917E0626
:100F100090917F060E94040E66E271E080917E0649
:100F200090917F060E947C0349855A856B857C855C
:100F300080917E0690917F060E94040E63E271E02C
:100F400080917E0690917F060E947C03B501A401EA
:100F500080917E0690917F060E94040E60E271E00F
:100F600080917E0690917F060E947C03B301A201CE
:100F700080917E0690917F060E941F0E6EE171E0C7
:100F800080917E0690917F060E947C036091880488
:100F90007091890480917E0690917F060E94070ED1
:100FA0006BE171E080917E0690917F060E947C0348
:100FB0006A8D7B8D80917E0690917F060E94070E40
:100FC000111113C068E171E080917E0690917F0657
:100FD0000E947C03ED81FE81E85FFC4F608180917F
:100FE0007E0690917F060E94690EC114D104E1042F
:100FF000F104C1F065E171E080917E0690917F0679
:101000000E947C036E897F89888D998DA701960146
:101010000E948919BA01A90180917E0690917F06EC
:101020000E94040E80917E0690917F06A1960FB6D5
:10103000F894DEBF0FBECDBFDF91CF911F910F910E
:10104000FF90EF90DF90CF90BF90AF909F908F90E8
:101050007F906F905F904F903F902F900C94B503CE
:10106000A1960FB6F894DEBF0FBECDBFDF91CF9132
:101070001F910F91FF90EF90DF90CF90BF90AF90B6
:101080009F908F907F906F905F904F903F902F90A8
:1010900008952F923F924F925F926F927F928F921C
:1010A0009F92AF92BF92CF92DF92EF92FF920F93F7
:1010B0001F93CF93DF936C014A015B018091F90488
:1010C00090E0029664E170E00E947519FC0120E056
:1010D00030E040E0C4E1D0E0CF01820F931FBE01B9
:1010E0000E947519DC01A656BD4F8C9190E08C15BD
:1010F0009D0509F44F5F2F5F3F4F2431310561F7A4
:10110000442309F4D7C01F0163E171E080917E069A
:1011100090917F060E947C03F601EE0FFF1FE65BB5
:10112000F94F6081718180917E0690917F060E94C7
:10113000510E61E171E080917E0690917F060E94E0
:101140007C03E12CF12C21E0C701820D931D64E1A9
:1011500070E00E9475198C01FC01E656FD4F8081FC
:1011600090E0C816D90609F085C0E801CC0FDD1F54
:10117000CC0FDD1F211120C0FE01E65BFD4F8081F9
:101180009181A281B381FE01E650FE4F40815181E1
:1011900062817381840F951FA61FB71F8415950563
:1011A000A605B70508F45FC06EE071E080917E0689
:1011B00090917F060E947C03F801EE0FFF1FEE5214
:1011C000FE4F6081718180917E0690917F060E9422
:1011D000070E6CE071E080917E0690917F060E9480
:1011E0007C03FE01E65BFD4F40815181628173818A
:1011F000481959096A097B0980917E0690917F06FA
:101200000E941F0E6AE071E080917E0690917F0639
:101210000E947C03FE01E650FE4F408151816281B5
:10122000738180917E0690917F060E94040E68E093
:1012300071E080917E0690917F060E947C03F80108
:10124000E254FE4F608180917E0690917F060E945D
:10125000690EF801E655FE4F608180917E069091FF
:101260007F060E947503C65BDD4F488059806A8007
:101270007B8020E08FEFE81AF80A84E1E816F10499
:1012800009F062CF80917E0690917F06DF91CF9129
:101290001F910F91FF90EF90DF90CF90BF90AF9094
:1012A0009F908F907F906F905F904F903F902F9086
:1012B0000C94B503DF91CF911F910F91FF90EF90A8
:1012C000DF90CF90BF90AF909F908F907F906F9066
:1012D0005F904F903F902F9008950F931F93CF935F
:1012E000DF93EC0166E071E080917E0690917F06CD
:1012F0000E947C038E01000F111FF801E65BF94F7D
:101300006081718180917E0690917F060E94510ECE
:10131000FE01EB5CF94F208180917E0690917F0663
:10132000222329F0213031F46EEF70E005C065EF23
:1013300070E002C062EF70E00E947C03CD5DD94F87
:101340008881882341F06AEE70E080917E0690915A
:101350007F060E947C0364EE70E080917E0690918F
:101360007F060E947C03F801E150FA4F6081718191
:1013700080917E0690917F06DF91CF911F910F9112
:101380000C94070E62EE70E080917E0690917F06CD
:101390000E947C03609102017091030180917E069E
:1013A00090917F060E94510E60EE70E080917E0663
:1013B00090917F060E947C03609100017091010171
:1013C00080917E0690917F060C94570ECF92DF920B
:1013D000EF92FF926EED70E080917E0690917F0615
:1013E0000E947C0360910E0170910F0180911001A9
:1013F0009091110128EEC22E23E0D22EE12CF12C87
:10140000A70196010E948919BA01A90180917E065F
:1014100090917F060E94040E6CED70E080917E0634
:1014200090917F060E947C0360910A0170910B01EC
:1014300080910C0190910D01A70196010E948919DC
:10144000BA01A90180917E0690917F060E94040E48
:101450006AED70E080917E0690917F060E947C0389
:101460006091060170910701809108019091090136
:10147000A70196010E948919BA01A90180917E06EF
:1014800090917F060E94040E68ED70E080917E06C8
:1014900090917F060E947C03609104017091050188
:1014A00080917E0690917F06FF90EF90DF90CF9025
:1014B0000C940D0E0F931F93CF93DF93C6ECD0E0E7
:1014C000FE01649180917E0690917F060E947503D3
:1014D0002196F0E0C73DDF0799F761EC70E080915D
:1014E0007E0690917F060E947C03CCEBD0E0FE014B
:1014F000649180917E0690917F060E9475032196EB
:10150000F0E0C03CDF0799F761EB70E080917E0668
:1015100090917F060E947C03CCE9D0E000EB10E0C4
:10152000FE01649180917E0690917F060E94750372
:1015300021960C171D07A1F7DF91CF911F910F91F5
:101540000895CF92DF92EF92FF920F931F93CF9364
:10155000DF930E948B106B017C0180917E0690913D
:101560007F060E94B5030E945A0A69E471E08091E7
:101570007E0690917F060E947C0306E611E0C0E0A3
:1015800081E0F801219131918F0137FD12C0811165
:1015900008C067E471E080917E0690917F060E940A
:1015A0007C036C2F80917E0690917F060E94690ECD
:1015B00080E0CF5FC63129F76CE371E080917E0651
:1015C00090917F060E947C0369E371E080917E0622
:1015D00090917F060E947C03B701A60180917E0650
:1015E00090917F060E94040E67E371E080917E0671
:1015F00090917F060E947C03609188047091890419
:1016000080917E0690917F060E94070E64E371E050
:1016100080917E0690917F060E947C034091840415
:1016200050918504609186047091870480917E06B4
:1016300090917F060E94040E62E371E080917E0625
:1016400090917F060E947C036091820470918304D4
:1016500080917E0690917F060E94070E80917E0603
:1016600090917F060E94B5030E94E6090E94C2097C
:1016700060E371E080917E0690917F060E947C037A
:101680006091580580917E0690917F060E94700EB1
:101690000AE416E0C0E0D0E0F801819191918F0159
:1016A00097FD09C0CE010E946D0980917E06909140
:1016B0007F060E94B5032196C231D10569F7DF91FB
:1016C000CF911F910F91FF90EF90DF90CF900895F1
:1016D000CF93DF93C4E9D0E0FE01649180917E0650
:1016E00090917F060E9475032196F0E0CB39DF07C9
:1016F00099F7DF91CF9108954F925F926F927F9209
:101700008F929F92AF92BF92DF92EF92FF920F93D0
:101710001F93CF93DF93D62E682F70E08B01000FBD
:10172000111F000F111FF801E65EFC4F80809180B1
:10173000A280B38029013A01481859086A087B0839
:10174000530142019091F9049F5F9093F9049091A5
:10175000F904943110F01092F904E091F904F0E0EA
:10176000A091A801B091A901ED012196D093A90102
:10177000C093A801EE0FFF1FEE52FE4FB183A0836E
:10178000E091F904F0E0E656FD4F8083E091F90422
:10179000C801865E9C4F7C01EC0188819981AA81F9
:1017A000BB81D4E0ED9FF0011124E65BFD4F808307
:1017B0009183A283B383E091F90484E0E89FF00170
:1017C0001124E650FE4F80829182A282B382A091C2
:1017D000F904B0E0FB01EA50FD4F8081A254BE4FF6
:1017E0008C93CB01880F991FDC01A150BA4F0D904B
:1017F000BC91A02D2D01612C712CEB01CB5CD94F3C
:1018000084149504A604B704B0F4D7012D933D9336
:101810004D935C93139770816881761372C0DC01DD
:10182000A357BB4F8D919C911197019611969C9354
:101830008E9362E567C0A081B881CB018A569E4F26
:10184000AB135AC0EC01B881AB1709F442C0D80100
:10185000AF54BB4F4D905D906D907C901397DFEF30
:101860004D1A5D0A6D0A7D0A4D925D926D927C92D1
:101870001397D801AE59BC4F2D933D934D935C9374
:101880001397DB01A059BB4FCC91C1110FC0E801E8
:10189000C655DC4F288339834A835B83C1E0CC93F0
:1018A000DB01A25ABB4F6C916F5F6C93D801A255BC
:1018B000BD4F4D905D906D907C901397840C951C5E
:1018C000A61CB71C8D929D92AD92BC92139763E4B7
:1018D00014C0D801A255BD4F4D905D906D907C9085
:1018E0001397840C951CA61CB71C8D929D92AD92EB
:1018F000BC92139760E501C067E47081DC017C93C2
:1019000001C068E5A091F904B0E0A655BE4F6C9304
:10191000D801A65EBC4F2D933D934D935C931397D6
:10192000D082DF91CF911F910F91FF90EF90DF90C8
:10193000BF90AF909F908F907F906F905F904F90EF
:101940000895BF92CF92DF92EF92FF920F931F9371
:10195000CF93DF93C82F0E948B106B017C018C2FDB
:1019600090E0FC01EE0FFF1FE350FC4FA591B491F6
:101970000C91DC01A95BB94F1C91FC01EE0FFF1F1C
:10198000E65DFE4F0190F081E02D208110271223AB
:101990000C93112339F1FC01EB5EFE4FC081D1E0C5
:1019A000FC01EE5EFE4FB080BC16E0F08D2F81236F
:1019B000B1F0EC2FF0E0EE0FFF1FEA59FE4F01905F
:1019C000F081E02D1E161F0654F461E09D2F902338
:1019D00009F460E0A70196018E2F0E947C0BDD0FB9
:1019E000CF5FE2CFDF91CF911F910F91FF90EF90EA
:1019F000DF90CF90BF9008951F920F920FB60F9275
:101A000011242F933F934F935F936F937F938F9303
:101A10009F93AF93BF93EF93FF9382E00E94A10C3B
:101A2000FF91EF91BF91AF919F918F917F916F91B6
:101A30005F914F913F912F910F900FBE0F901F908C
:101A400018951F920F920FB60F9211242F933F9368
:101A50004F935F936F937F938F939F93AF93BF93B6
:101A6000EF93FF9381E00E94A10CFF91EF91BF9152
:101A7000AF919F918F917F916F915F914F913F9126
:101A80002F910F900FBE0F901F9018951F920F92DD
:101A90000FB60F9211242F933F934F935F936F9341
:101AA0007F938F939F93AF93BF93EF93FF9380E0C8
:101AB0000E94A10CFF91EF91BF91AF919F918F91E7
:101AC0007F916F915F914F913F912F910F900FBE3A
:101AD0000F901F9018950E94D4198F929F92AF92E9
:101AE000BF92EF92FF920F931F93CF93DF93CDB7E7
:101AF000DEB7A1970FB6F894DEBF0FBECDBF7C0155
:101B0000FA01CB0119A2223008F42AE08E010F5D00
:101B10001F4F822E912CA12CB12CBF01A501940145
:101B20000E948919F901CA01015011096A3014F49F
:101B3000605D01C0695CD8016C93232B242B252B9D
:101B400061F7B801C7010E94A003A1960FB6F894EF
:101B5000DEBF0FBECDBFDF91CF911F910F91FF90E0
:101B6000EF90BF90AF909F908F900895833081F059
:101B700028F4813099F08230A1F008958730A9F0DF
:101B80008830B9F08430D1F4809180008F7D03C01B
:101B9000809180008F7780938000089584B58F773F
:101BA00002C084B58F7D84BD08958091B0008F7789
:101BB00003C08091B0008F7D8093B00008953FB73F
:101BC000F8948091850690918606A0918706B09141
:101BD000880626B5A89B05C02F3F19F00196A11DC8
:101BE000B11D3FBFBA2FA92F982F8827820F911DB3
:101BF000A11DB11DBC01CD0142E0660F771F881FFA
:101C0000991F4A95D1F708952AE00C946D0DAB0108
:101C100060E070E02AE00C946D0D0F931F93CF935A
:101C2000DF93EC010E94070E8C01CE010E94B503E8
:101C3000800F911FDF91CF911F910F910895CF9247
:101C4000DF92EF92FF920F931F93CF93DF9377FF73
:101C50001DC06A017B01EC016DE20E9475038C01DD
:101C600044275527BA014C195D096E097F092AE0FE
:101C7000CE010E946D0D800F911FDF91CF911F91BA
:101C80000F91FF90EF90DF90CF9008952AE0DF91C1
:101C9000CF911F910F91FF90EF90DF90CF900C9418
:101CA0006D0DAB01770F660B770B0C941F0E0F9326
:101CB0001F93CF93DF93EC010E94510E8C01CE0154
:101CC0000E94B503800F911FDF91CF911F910F915B
:101CD0000895462F50E060E070E02AE00C946D0D0E
:101CE0000F931F93CF93DF93EC010E94690E8C0139
:101CF000CE010E94B503800F911FDF91CF911F91FC
:101D00000F910895843058F40E94680B6FE674E0D8
:101D100080917E0690917F060E947C03B2C0209144
:101D20006E0630916F06C901019780319E4038F0F0
:101D30000E94680B60916E0670916F0650C0A8EE0D
:101D4000B3E00E94B11960930E0170930F0180936C
:101D50001001909311012091700630917106C90114
:101D6000019780319E4038F00E94680B60917006A8
:101D70007091710634C0A8EEB3E00E94B11960936F
:101D80000A0170930B0180930C0190930D01209137
:101D900072063091730621318EE0380738F00E94C8
:101DA000680B609172067091730619C0A8EEB3E0DB
:101DB0000E94B11960930601709307018093080196
:101DC000909309018091740690917506853691056E
:101DD00060F00E94680B60917406709175068091A6
:101DE0007E0690917F060C940D0E909305018093D2
:101DF00004016BE574E080917E0690917F060E945D
:101E00007C0360916E0670916F0680917E069091C2
:101E10007F060E94070E69E574E080917E0690912E
:101E20007F060E947C03609170067091710680911C
:101E30007E0690917F060E94070E67E574E0809110
:101E40007E0690917F060E947C03609172067091DD
:101E5000730680917E0690917F060E94070E65E5CD
:101E600074E080917E0690917F060E947C036091D1
:101E700074067091750680917E0690917F060E948F
:101E8000070E80917E0690917F060C94B5038230F8
:101E900058F40E94680B60E574E080917E06909192
:101EA0007F060E947C0353C080916E0690916F065E
:101EB0009C01215031092F3F334038F00E94680BBC
:101EC00060916E0670916F0614C090930301809329
:101ED000020180917006909171069C012150310998
:101EE0002F3F334060F00E94680B60917006709144
:101EF000710680917E0690917F060C940D0E909352
:101F000001018093000164E374E080917E0690916A
:101F10007F060E947C0360916E0670916F0680912F
:101F20007E0690917F060E94070E62E374E0809126
:101F30007E0690917F060E947C03609170067091EE
:101F4000710680917E0690917F060E94070E809117
:101F50007E0690917F060C94B50387E480937C0005
:101F600080917A00806480937A0080917A0086FD67
:101F7000FCCF809178002091790090E0922B089519
:101F80001F93CF93DF93E6E9F3E09491EAEAF3E05D
:101F9000D491E5E0F4E0C491CC23D1F0182F99233B
:101FA00019F0892F0E94B60DEC2FF0E0EE0FFF1F05
:101FB000E657FC4FA591B4919FB7F894111104C056
:101FC0008C91D095D82302C0EC91DE2BDC939FBF7F
:101FD000DF91CF911F910895CF93DF93282F30E0A9
:101FE000F901EC56FC4F8491F901E855FC4FD4916E
:101FF000F901ED5FFB4FC491CC2391F081110E9458
:10200000B60DEC2FF0E0EE0FFF1FE750FC4FA5914F
:10201000B491EC91ED2381E090E021F480E002C0E6
:1020200080E090E0DF91CF910895CF93DF9390E02F
:10203000FC01E855FC4F2491FC01ED5FFB4F8491BE
:10204000882361F190E0880F991FFC01E058FC4F54
:10205000C591D491FC01E657FC4FA591B491611153
:1020600009C09FB7F8948881209582238883EC91DA
:102070002E230BC0623061F49FB7F8948881322F11
:10208000309583238883EC912E2B2C939FBF06C021
:102090008FB7F894E8812E2B28838FBFDF91CF91E3
:1020A00008958F929F92AF92BF92CF92DF92EF925C
:1020B000FF926B017C010E94DF0D4B015C01C1149A
:1020C000D104E104F104F1F00E94DF0DDC01CB0149
:1020D00088199909AA09BB09883E9340A105B10551
:1020E00070F321E0C21AD108E108F10888EE880EE9
:1020F00083E0981EA11CB11CC114D104E104F104B9
:1021000019F7DDCFFF90EF90DF90CF90BF90AF90A9
:102110009F908F9008952FB7F894609181067091E9
:10212000820680918306909184062FBF08957F9246
:102130008F929F92AF92BF92CF92DF92EF92FF92D7
:102140000F931F93CF93DF93782E0E948B10AB01D8
:10215000BC01C0906E06D0906F0685E18C1558F0DA
:102160005601BB24F501EE0FFF1FEA59FE4F008117
:10217000118117FF1EC00E94680B67E174E0809117
:102180007E0690917F060E947C036C2D80917E06D6
:1021900090917F06DF91CF911F910F91FF90EF906B
:1021A000DF90CF90BF90AF909F908F907F900C94D6
:1021B000700E11277801EE0CFF1CF701EE5BFE4F4D
:1021C000C081D181F701E65BF94F4F018081918198
:1021D000A816B906D1F0FE01FF27ED5FFB4FE49191
:1021E000E2508E2F90E0FC01EE0FFF1FE350FC4FFA
:1021F000A591B4912C91FC01E95BF94F2083C801B2
:102200000E942504F401B182A08280917006909111
:1022100071060297029788F00E94680B6EEC73E0DB
:1022200080917E0690917F060E947C036C2D8091A8
:102230007E0690917F060E94700EF801EB5CF94FCC
:1022400081E020917006309171062330310509F04C
:1022500080E08083C801805D9E4F6C01F801ED5DD8
:10226000F94F5F01F2E0F71590F4809172069091BA
:102270007306892B61F0F6018081811108C062E04C
:102280008C2F0E94151081E0F501808306C060E06C
:102290008C2F0E941510F5011082F3E0F71530F431
:1022A0008091740690917506009711F482E090E099
:1022B000F701E150FA4F91838083F601808181110B
:1022C00023C0DD27FE01E855FC4F8491FE01ED5F40
:1022D000FB4FC491CC23B1F1C250AC2FB0E0AA0F98
:1022E000BB1FA65DBE4F0D90BC91A02DEC91E82BBD
:1022F000EC932091680081E090E001C0880FCA95BE
:10230000EAF7822B809368006CEB73E080917E0685
:1023100090917F060E947C03C8010E946D09809104
:102320007E0690917F06DF91CF911F910F91FF90D4
:10233000EF90DF90CF90BF90AF909F908F907F9065
:102340000C94B5030E94680B67EC73E080917E06E5
:1023500090917F06DF91CF911F910F91FF90EF90A9
:10236000DF90CF90BF90AF909F908F907F900C9414
:10237000B9031F920F920FB60F9211242F933F9320
:102380008F939F93AF93BF93809181069091820624
:10239000A0918306B09184063091800623E0230F3C
:1023A0002D3720F40196A11DB11D05C026E8230F8D
:1023B0000296A11DB11D2093800680938106909303
:1023C0008206A0938306B09384068091850690913F
:1023D0008606A0918706B09188060196A11DB11DC1
:1023E0008093850690938606A0938706B09388060F
:1023F000BF91AF919F918F913F912F910F900FBE01
:102400000F901F901895E9E5F5E01382128288EE8F
:1024100093E0A0E0B0E084839583A683B7838CE14A
:1024200091E09183808385EC90E09587848784ECAC
:1024300090E09787868780EC90E0918B808B81EC91
:1024400090E0938B828B82EC90E0958B848B86EC72
:1024500090E0978B868B118E128E138E148E0895BA
:10246000CF93DF93CDB7DEB727970FB6F894DEBFD3
:102470000FBECDBF789484B5826084BD84B5816081
:1024800084BD85B5826085BD85B5816085BD80913F
:102490006E00816080936E001092810080918100B7
:1024A00082608093810080918100816080938100AF
:1024B000809180008160809380008091B100846071
:1024C0008093B1008091B00081608093B0008091D2
:1024D0007A00846080937A0080917A008260809391
:1024E0007A0080917A00816080937A0080917A00EE
:1024F000806880937A001092C100E0916905F091A4
:102500006A0582E08083E0916505F091660510829E
:10251000E0916705F091680583E38083109271056F
:10252000E0916D05F0916E0586E08083E0916B058A
:10253000F0916C05808180618083E0916B05F09162
:102540006C05808188608083E0916B05F0916C055B
:10255000808180688083E0916B05F0916C058081BB
:102560008F7D808364EF71E080E090E00E945110E5
:10257000789489E595E00E94B50389E595E090930C
:102580007F0680937E0610928904109288040E9430
:102590008B106093F6057093F7058093F805909380
:1025A000F9050E94940461E082E00E9415100E94E7
:1025B000A10A18EE212E13E0312E412C512C0E943D
:1025C0008B100091F6051091F7052091F8053091D8
:1025D000F905601771078207930750F4209188046A
:1025E000309189042F5F3F4F3093890420938804F2
:1025F0006093F6057093F7058093F8059093F905BD
:1026000089E595E00E94C402892B09F4AAC289E5F4
:1026100095E00E94A202D82EBCE28B2E881119C030
:10262000E0918C04E73008F09CC281E08E0F80932B
:102630008C04F0E0EE0FFF1FE259F94F80918A04FD
:1026400090918B049183808310928B0410928A0462
:1026500088C280ED8D0D8A30A8F420918A043091D3
:102660008B04EAE09E2E929EC001939E900D112451
:10267000C0978D0D911DD7FC9A9590938B048093F4
:102680008A046FC28FE98D0D8A3108F06AC2809189
:102690005805882309F44BC0E0918C04F0E0EE0F5C
:1026A000FF1FE259F94F80918A0490918B04918326
:1026B00080836DEB72E089E595E00E947C037EE605
:1026C000E72E76E0F72E00E010E080918C0490E099
:1026D00080179107A4F00115110531F06BEB72E042
:1026E00089E595E00E947C03F701619171917F017A
:1026F00089E595E00E94070E0F5F1F4FE6CF6D2D15
:1027000089E595E00E94750364EB72E089E595E048
:102710000E947C0360918C0470E06F5F7F4F89E5BD
:1027200095E00E94510E89E595E00E94B5038D2D3C
:10273000DD0C990BAA0BBB0BFC01E156F109E6314C
:10274000F10508F000C2EC5CFF4F0C94AB198091CE
:102750008C04E82FF0E0EE0FFF1FE259F94F2091B3
:102760008A0430918B04318320838F5F0E949710FD
:10277000EAC180918C04E82FF0E0EE0FFF1FE259D0
:10278000F94F20918A0430918B043183208300918A
:102790006E0610916F068F3F61F0063150F4F8011C
:1027A000FF27EE0FFF1FEA59FE4F8081918197FFAF
:1027B00005C00E94680B6EE572E046C49927FC01D3
:1027C000E05DFE4F2081211138C4FC01EE0FFF1F98
:1027D000EE5BFE4F208131813327F901E855FC4F34
:1027E0004491F901ED5FFB4F2491222309F41CC4AD
:1027F0002250A22FB0E0AA0FBB1FA65DBE4F0D90C6
:10280000BC91A02D3C91409543234C933C913111B8
:1028100014C46091680041E050E04A0102C0880C95
:10282000991C2A95E2F794012095262320936800AD
:1028300004C41A82198263E4CE0101960E948705BE
:1028400066E6CE0101960E94870567E6CE010196F5
:102850000E948705FAE46F2EF6E07F2EF30181E0F7
:102860002191319137FF8F5F06E0EE36F007C1F717
:102870008F5F8B83682FCE0101960E948705E090C1
:102880000401F090050160910601709107018091AB
:10289000080190910901A20191010E9489192C83DC
:1028A0003D834E835F8360910A0170910B0180919B
:1028B0000C0190910D01A20191010E948919490119
:1028C0005A0160910E0170910F0180911001909159
:1028D0001101A20191010E948919BA01A9010C817B
:1028E0001D81940169E4CE0101960E94A405209106
:1028F0000001309101014091020150910301E12C4E
:10290000F12C00E010E064E5CE0101960E94A405E0
:102910006FEF862E65E0962E73E2A72E76E0B72E37
:10292000E5E3CE2EE6E0DE2EF301419151913F0129
:1029300057FD14C0F401E080F180F501008110E042
:10294000F6018081811103C022E030E002C023E063
:1029500030E061E4CE0101960E94A405F2E08F0E02
:10296000911C0FEFA01AB00A1FEFC11AD10A2EE670
:10297000621626E07206C1F66DE372E089E595E025
:102980000E947C036B8189E595E00E94690E6AE3F1
:1029900072E089E595E00E947C0369817A8189E58E
:1029A00095E00E94570ECFC00E94A10ACCC0809132
:1029B0008C04E82FF0E0EE0FFF1FE259F94F209151
:1029C0008A0430918B04318320838F5F0E94820EB2
:1029D000BAC080918C04E82FF0E0EE0FFF1FE2599F
:1029E000F94F20918A0430918B0431832083209108
:1029F0006E0630916F062130310509F0A4C08F3F7B
:102A000009F4A1C064E372E013C30E9494049BC064
:102A10000E948B104B015C0169E272E080917E069E
:102A200090917F060E947C030E945A0A80917E0644
:102A300090917F060E94B5030E94E6090E94C20998
:102A400067E272E080917E0690917F060E947C038F
:102A50006091580580917E0690917F060E94700ECD
:102A60003AE4E32E36E0F32E00E010E0F701819126
:102A700091917F0197FD16C0C8010E946D0964E223
:102A800072E080917E0690917F060E947C03A501F2
:102A9000940161E0C8010E94DD05B501A401C801EF
:102AA0000E9449080F5F1F4F02311105F9F680E0BF
:102AB00090E00E94230400917E0610917F068334EB
:102AC00009F0BDC381E090E00E942304863609F03E
:102AD000B6C382E090E00E942304873609F0AFC3BA
:102AE000C1C280918C04E82FF0E0EE0FFF1FE25985
:102AF000F94F20918A0430918B04318320838F5FBA
:102B00000E94470F20C020918A0430918B0480914D
:102B10007E0690917F062F3F310588F4209358055B
:102B20006FE972E00E947C0360918A0470918B04CB
:102B300080917E0690917F060E940D0E04C069E789
:102B400072E00E94B90310928C0410928B041092D0
:102B50008A04EEE6F6E01192119206E0EE37F007F5
:102B6000D1F780916C0690916D0697FD36C180E09B
:102B70000E94C00F6AE070E080E090E00E94511077
:102B80000E94AD0F8C019093FE058093FD0581E0BE
:102B90000E94C00F6AE070E080E090E00E94511057
:102BA0000E94AD0F9093FC058093FB05801B910B59
:102BB00020910001309101012817390754F020912C
:102BC000020130910301821793070CF0C6C010E098
:102BD00001C011E08091FA05811709F4BEC010937D
:102BE000FA050E948B109B01AC01612F81E10E94CC
:102BF0007C0B809158058A3030F169E173E0809157
:102C00007E0690917F060E947C0361E170E08091D6
:102C10007E0690917F060E94510E67E073E08091DE
:102C20007E0690917F060E947C036091FA05809158
:102C30007E0690917F060E94690E80917E0690919B
:102C40007F060E94B503809158058A3008F485C03C
:102C500060E073E080917E0690917F060E947C0385
:102C600065E170E080917E0690917F060E94510E92
:102C700067EF72E080917E0690917F060E947C0350
:102C800061E170E080917E0690917F060E94510E76
:102C90006BEE72E080917E0690917F060E947C032D
:102CA00065E170E080917E0690917F060E94510E52
:102CB00067EE72E080917E0690917F060E947C0311
:102CC00062EE72E080917E0690917F060E947C0306
:102CD000612F80917E0690917F060E94690E67EDBC
:102CE00072E080917E0690917F060E947C03609145
:102CF000F90480917E0690917F060E94690E6EEC29
:102D000072E080917E0690917F060E947C03409144
:102D1000F5045091F6046091F7047091F8048091E5
:102D20007E0690917F060E94040E64EC72E0809112
:102D30007E0690917F060E947C036091AF047091A3
:102D4000B00480917E0690917F060E94070E8091CC
:102D50007E0690917F060E94B503809158058431CC
:102D6000E0F16EE773E080917E0690917F060E940D
:102D70007C036091FB057091FC0580917E0690912B
:102D80007F060E94510E6CE773E080917E06909161
:102D90007F060E947C036091FD057091FE05809185
:102DA0007E0690917F060E94510E69E773E0809144
:102DB0007E0690917F060E947C036091FB057091D6
:102DC000FC058091FD059091FE05681B790B8091B3
:102DD0007E0690917F060E94570E809158058A309A
:102DE00060F50E948B1000915405109155052091BB
:102DF0005605309157054B015C01801A910AA20AD1
:102E0000B30AC0900E01D0900F01E0901001F09035
:102E100011018C149D04AE04BF0408F0D6C0C0900C
:102E20000A01D0900B01E0900C01F0900D01EAE452
:102E3000F6E0ACE0B5E040E0C1C05AE4A52E56E0B3
:102E4000B52E6AEFE62E64E0F62E72E4C72E71E02E
:102E5000D72E00E010E0F501819091905F011814E9
:102E600019040CF085C0F6016080862D0E94EC0FDD
:102E7000782EF7018081781609F47AC0708262E7B3
:102E800073E080917E0690917F060E947C03B401DE
:102E900080917E0690917F060E94510E66E673E057
:102EA00080917E0690917F060E947C03662D809122
:102EB0007E0690917F060E94690E64E673E0809121
:102EC0007E0690917F060E947C0367E573E0809107
:102ED0007E0690917F060E947C03672D80917E067E
:102EE00090917F060E94690E6CE473E080917E06EB
:102EF00090917F060E947C036091F90480917E0688
:102F000090917F060E94690E63E473E080917E06D3
:102F100090917F060E947C03F801EE0FFF1FEE0FD9
:102F2000FF1FEF54FB4F408151816281738180917B
:102F30007E0690917F060E94040E69E373E0809103
:102F40007E0690917F060E947C03F801EE0FFF1F22
:102F5000E357FB4F6081718180917E0690917F06DF
:102F60000E94070E80917E0690917F060E94B50315
:102F70000F5F1F4FFFEFEF1AFF0A22E0C20ED11CB6
:102F80000231110509F067CF2CCF0D911D912D91C4
:102F90003C9113974B015C01801A910AA20AB30A73
:102FA0008C149D04AE04BF0408F041E014962EE694
:102FB000A22E26E0B22EAE16BF0629F02191319145
:102FC00037FDF4CFE2CF442361F10E948B104B0117
:102FD0005C018AE4E82E86E0F82E00E010E0F701BC
:102FE000819191917F0197FD0FC0A501940160E04F
:102FF000C8010E94DD0580915805853028F0B50193
:10300000A401C8010E9449080F5F1F4F023111053A
:1030100031F78092540590925505A0925605B092D2
:1030200057050E946B03CBCA0E94680B67E572E0EC
:1030300080917E0690917F0684CD40E050E0BA01F9
:103040000E9425046CE472E080917E0690917F06D8
:103050000E947C03602F80917E0690917F060E94E3
:10306000700E71CD83E090E00E942304682EF4E19D
:10307000F81718F463ED71E0E4C0C8010E94B503CD
:1030800061EC71E080917E0690917F060E947C0346
:1030900080E090E00E942304682F80917E0690914A
:1030A0007F060E94750381E090E00E942304682F50
:1030B00080917E0690917F060E94750382E090E0E9
:1030C0000E942304682F80917E0690917F060E94C3
:1030D000750368EB71E080917E0690917F060E94F7
:1030E0007C0383E090E00E942304682F70E08091CD
:1030F0007E0690917F060E94510E80917E069091EF
:103100007F060E94B503712C04E010E0671409F4F7
:103110009BC0C8010E9423048B83C80101960E94B2
:103120002304F82EC80102960E942304882E912CB5
:10313000982C88248F0C911CC80103960E942304AC
:10314000F82EC80104960E942304A82EB12CBA2C94
:10315000AA24AF0CB11CC80105960E942304F82EC6
:10316000C80106960E942304C82ED12CDC2CCC2446
:10317000CF0CD11CC80107960E942304F82EC80169
:1031800008960E94230490E0982F88279C012F0D19
:10319000311D7901075F1F4F6FEA71E080917E0654
:1031A00090917F060E947C036B8180917E069091B6
:1031B0007F060E9475036DEA71E080917E06909112
:1031C0007F060E947C03B40180917E0690917F0669
:1031D0000E94070E6BEA71E080917E0690917F0657
:1031E0000E947C03B50180917E0690917F060E942B
:1031F000070E69EA71E080917E0690917F060E9439
:103200007C03B60180917E0690917F060E94070E96
:1032100067EA71E080917E0690917F060E947C03B0
:10322000B70180917E0690917F060E94070E8091E3
:103230007E0690917F060E94B503739467CF6EEE71
:1032400071E0C8010E94B90362E172E080917E06DC
:1032500090917F060E947C03C0905405D090550544
:10326000E0905605F090570580910E0190910F0166
:10327000A0911001B0911101C80ED91EEA1EFB1ECB
:103280000E948B1046015701861A970AA80AB90AAC
:10329000B501A40180917E0690917F060E94040EE4
:1032A00064E072E080917E0690917F060E947C032C
:1032B00080917E0690917F060E94B50344CCF999D7
:1032C000FECF92BD81BDF89A992780B50895262F2B
:1032D000F999FECF1FBA92BD81BD20BD0FB6F894FB
:1032E000FA9AF99A0FBE0196089597FB072E16F4E5
:1032F000009407D077FD09D00E94C01907FC05D0C3
:103300003EF4909581959F4F0895709561957F4FFC
:103310000895A1E21A2EAA1BBB1BFD010DC0AA1F16
:10332000BB1FEE1FFF1FA217B307E407F50720F02E
:10333000A21BB30BE40BF50B661F771F881F991FA9
:103340001A9469F760957095809590959B01AC01F2
:10335000BD01CF010895EE0FFF1F0590F491E02D00
:103360000994A29FB001B39FC001A39F700D811D5E
:103370001124911DB29F700D811D1124911D08957E
:10338000AA1BBB1B51E107C0AA1FBB1FA617B7078B
:1033900010F0A61BB70B881F991F5A95A9F78095A7
:1033A0009095BC01CD01089581E090E0F8940C94D3
:0633B000D919F894FFCFCB
:1033B6006E0064000200D007000060EA000030756D
:1033C60000000D1307080E0000000000FC02650255
:1033D60093024903C402A202B6026B006C006D00A0
:1033E60000000000000000000000000000000000D7
:1033F600000103000400050006000700080009009C
:103406000A000B000C000E000F0010001100120045
:10341600130014001500FFFFFFFFFFFF000001006F
:103426000200030004000500060007000800FFFF75
:1034360009000A000B000C000D000E000F00100022
:0634460011000D0A000058
:00000001FF
